:020000040000FA
:1000000064008B01442882000000080020344D3435
:1000100048347A34203400342034203420340034FE
:1000200055345334423400344C3453344234003465
:100030005034523447340034433441344C34003467
:1000400046344D3432342E34303430343934203464
:1000500000342D34203456344B3433344234483455
:10006000523400342034203420344F347634653414
:10007000723420340034523461346E346734653461
:1000800020342034203400348B218501860105146E
:10009000682120300E21851C812129300E2141212B
:1000A00041218421061A8B28FD30C200FF30C30095
:1000B000BF30C4000030C5009421BC211C300E218B
:1000C0008721061B6B28C40A031D6A28C30A031D67
:1000D0006A28C20A7C28861B7C28FF30C407031CC0
:1000E0007528C30A031D7528C20AFF30C307031C05
:1000F0007A28C20AFF30C207061E5C284121061E6C
:100100005C284208BE004308BF004408C000450800
:10011000C100103002221030D8213E08C2003F0832
:10012000C3004008C4004108C5008721A901AF11E0
:10013000AF12061AB1284121061AB12894213A08B3
:10014000BE003B08BF003C08C0003D08C100BC2108
:1001500018300E218721061E9E284121061E9E284A
:10016000AF16861FB628061FBF28C228061FB9284B
:10017000BB280030C328AF15A9090430C328AF1528
:100180000830C3280C30AF1AC728D821C82802224B
:100190009421861ECC28F820DD20BA1FD128F82013
:1001A000A909BC21AF19D6280C30DB282918DA2878
:1001B0001030DB2814300E218B284108BD07031CAA
:1001C000E828BC0A031DE828BB0A031DE828BA0A70
:1001D0004008BC07031CF028BB0A031DF028BA0A1C
:1001E0003F08BB07031CF528BA0A3E08BA070800F7
:1001F000BA09BB09BC09BD09BD0A031D0629BC0A11
:10020000031D0629BB0A031D0629BA0A0800082196
:10021000BA0CBB0CBC0CBD0CBA130800AE002E0807
:100220000320FF39031905282921AE0A0F294208A6
:10023000B6004308B7004408B800B80F1D29B12123
:10024000B70F1D29B60F1D29003485112D290F392F
:10025000303EAD006D222D088515AC002C0E3121ED
:100260002C080F3986000515000005114230B60034
:10027000B60B382900340A30B7003621B70B3D29B8
:1002800000340301B8003B21B80B4329003420306F
:10029000AA00A401A501A601A701A8012430840099
:1002A0000530AB00333080078019F039801B0F39DF
:1002B0008002840AAB0B5229BD0DBC0DBB0DBA0DDB
:1002C000A80DA70DA60DA50DA40DAA0B4E2908007B
:1002D00041218511051103303121412103303121A4
:1002E00003303121023031212830252136210C30D4
:1002F00025213621063025213621013025213B21BB
:100300000034C03025213629013025213B295F22C8
:10031000023025213B2983163730810002308500C9
:10032000F03086008312080005120B118101BA011A
:10033000BB01BC01BD01051617210512000000001C
:10034000000000000000B1210108BC00831601126A
:10035000000001168312BD0301083C060319A629FB
:1003600008000B1DB9290B11BB0A031DB829BA0AD5
:10037000080000000000B8290721472125080F398F
:10038000031DC52920302921C6292721260E272112
:100390002E30292126082721270E2721270827214B
:1003A000280E272128082721851C812106300E29A7
:1003B00089000C3A0319EB29E621BE00E521BF00B4
:1003C000E521C000E521C1000800890A8316081450
:1003D0008312080808000430D8213E08BA003F08FC
:1003E000BB004008BC004108BD000830D821DD201A
:1003F00008213A08BE003B08BF003C08C0003D0889
:10040000C100080089003E080D223F080C22400868
:100410000C2241080C220800890A8800831608155E
:1004200055308900AA30890088148818152A0812C6
:1004300083120800FE30B8001D30B700C030B6008F
:1004400005100514B60F202AB70F202AB80F202A4E
:100450000800B200030EB3000408B40057306D2248
:100460003D306D223208632220306D2220306D2213
:1004700053306D2252306D223D306D22330863229D
:100480005F2284010008632220306D22840A040860
:100490000F39031D4D2A5F22522A0339031D522AA8
:1004A00020306D220408803A031D422A5F225F2219
:1004B00034088400330E8300B20E320E08000D3073
:1004C0006D220A306D2AB500350E672235080F39C6
:1004D000F63E031C6C2A073E3A3EB0000830B100DD
:1004E0000510E730013E031D722AB00C03187A2A6A
:1004F00005107B2A0514B10B712AE730013E031D5C
:0E0500007E2A0514CD30013E031D832A08001B
:02400E00F23F7F
:1042000000000000000000000000000000000000AE
:10421000000000000000000000000000000000009E
:08422000FD00FF00BF000000DB
:00000001FF
